:020000040000FA
:020000003528A1
:080008000428851C0D28051CCD
:100010001328051D19281F20052805128516851887
:1000200005281F200F2805128512051805281F20F6
:10003000152805168516851805281F201B2802304F
:10004000A5007F30A400A50B26282A282B20A40B6E
:100050002628212808000130A000C830013C003CBF
:10006000031D2E28A00B2D280800831285018B016B
:100070000730990000309F00831600309F008C01EC
:10008000960195010F3081000730850083128501AC
:100090000330A300FF3085001F20003085001F20A3
:0A00A000A30B4A2800308500052854
:02400E00843FED
:024200000800B4
:00000001FF
